:020000040000FA
:100000005E288207003400340034013400340034A8
:1000100000340A34003400340034643400340034D2
:100020000334E8340034003427341034003401340D
:100030008634A03400340F344234403400349834D1
:100040009634803482070B340A340934073406347A
:100050000534033402348207503449344334453480
:100060004C34673465346E3400342034563465348F
:10007000723432342E3431346634003442346134D4
:100080006E34643420340034553470346434613454
:1000900074346534003449346E3469347434423411
:1000A00061346E346434003420344B3448347A3450
:1000B0000034433441344C34203400348B01073055
:1000C0009F009801831698018C019F018113FF30D6
:1000D000850086018312A901AA01AB01AC01AD0123
:1000E000742274228E22AE2237308400F0019E23C7
:1000F000C601CA010508C50003304505C400451EF8
:10010000FB21D1015330DC000030CD000301E2219E
:100110000430F000B623D200BD20D7214523123091
:10012000B4222A23BF23F92273222E214A1E9A28A1
:10013000A3209528C6189E281221A028C920E820AF
:10014000F92273229528FF305C078400C618AE2878
:100150008003801FB4280D308000B428800A0E3040
:100160000002031CB428800145231230B4222A2344
:10017000BF23BD20F922732208005C08FF3E8400E3
:1001800005300007000700070007F000840A9E23DF
:100190000800CC015C0884002E0880070330C800EA
:1001A000E220840384032F0880070230C800E22085
:1001B000840330088007840A031CDF28800A310882
:1001C000800708004C0D840A8007C80BE22808004D
:1001D00003305C07840002300002031C1129031D58
:1001E0000429840362300002031C1129031D042921
:1001F00084035A300002031C1129031D04298403BF
:1002000000300002031C11295C08840000308000CB
:10021000840A5A308000840A62308000840A0230E6
:10022000800008002221C92003305C078400801F61
:1002300020298001840380018403800184038001DC
:1002400022210800AE09AF09B009B109AE0F2D296E
:10025000AF0F2D29B00F2D29B10A08006021050824
:10026000C500D42305084506031D2E290330450586
:10027000C300440603192E290310C40D4308C40605
:1002800044080239C7004606C601C4184F2943086E
:10029000C400D00350182E29D0182E295829023016
:1002A000C6004308C400D00A50182E29D0182E29A1
:1002B0004308C400C5195E294A165F294A1208007E
:1002C000CA18C029051DC129051A7D29851DA22925
:1002D0002030CB004A10CB23051A7B29851DA2298B
:1002E000051DC129CB03031D6B290130E221043018
:1002F000CB004A146B2901309E294A1E8329851D93
:10030000C029CA01C0298519C029CA198B292030E2
:10031000CB004A10CA15CB2385199D29051EA22999
:10032000CB0303199629CA19C0298B29CA11FF309A
:10033000E2210430CB004A148B29FF304A18BF2930
:10034000E221BF294030CB00CB23051AC0298519F3
:10035000C029CB03031DA4294A1EB82982234523A3
:100360001830B422BF2345231F30B422BD23BE2939
:10037000892345231830B4222A23BD23F922CA0138
:100380000800CB23051ECA16051DC129CA1ECA298D
:10039000D721D329511CD02951105330DC00D32947
:1003A00051145830DC00CA01F9227322C0295308C5
:1003B000D8005408D9005508DA005608DB00520866
:1003C000D70008004D070739CD002220CE00EA21D2
:1003D000F92208000430C800313084004D08CC00F8
:1003E0000310CC0DCC0D4C08012080008403CC0AF6
:1003F000C80BF3290800CA148030D3009630D4000B
:100400009830D5000030D600F9228C3060232D3092
:10041000B42273222E21B101B001AF010530AE002C
:100420004519142A8030AE000000C618182A22216F
:100430002E08B707031C212AB80F212AB90F212A39
:10044000BA0A2F08B807031C282AB90F282ABA0AA3
:100450003008B907031C2D2ABA0A3108BA07051E4D
:10046000092AF001373084009523CA100800A90139
:10047000AA01AB01AC01AD012030B4003708BB00CC
:100480003808BC003908BD003A08BE005C0884008A
:1004900003103B1C652A0008AA07031C542AAB0F53
:1004A000542AAC0F542AAD0A840A0008AB07031C77
:1004B0005C2AAC0F5C2AAD0A840A0008AC07031C56
:1004C000622AAD0A840A0008AD07AD0CAC0CAB0C77
:1004D000AA0CA90CBE0CBD0CBC0CBB0C5C08B40B6C
:1004E000472AAD0108003722293084000008B600F1
:1004F0000830B500B60C031C812A861506150611B6
:10050000842A861106150611B50B7A2A840A2E3024
:100510000402031C762A861786130800C8230330BA
:1005200086000616C8230612033086000616CB2363
:100530000612033086000616CB2306120230860010
:100540000616CE23061220306023083060230130C7
:100550006023063060230E30602308000030B42290
:100560000930B422BD230800CF002B20FF39031926
:10057000BD2A6423CF0A4F08B52A08002030B200F4
:10058000A401A501A601A701A8015C088400000838
:10059000A000840A0008A100840A0008A200840ABE
:1005A0000008A3000310A00DA10DA20DA30D0318B8
:1005B0002014A40DA50DA60DA70DA80DB203031DB3
:1005C000E22A080024308400EE22840AEE22840A03
:1005D000EE22840AEE22840AEE22D22A0330000799
:1005E000B300B319800030300007B300B31B8000A4
:1005F0000800BE220230602341305118423064238B
:1006000020306423270E0F39303E642327080F392A
:10061000303E64232C306423260E0F39303E642391
:1006200026080F39303E6423250E0F39303E6423EF
:100630002E30642325080F39303E6423240E0F39F1
:10064000303E642324080F39303E64232830B4221E
:1006500041230800A401A501520851185708CC00F5
:10066000CC0A0A304C02031C382BA400A50A3A2BF2
:100670004C08A4002508303E64232408303E64233F
:10068000080080304E046023080001306023080019
:100690008601831608308600831206138616FF3003
:1006A000C10006160608C00006120000000006166B
:1006B00000000612C10303195F2BC019512B08005B
:1006C000BF00C9010613672BBF0049140617482352
:1006D000860183160030860083128612061349189D
:1006E0000617F03086053F0E0F3986040616000007
:1006F0000612F03086053F080F3986040616000002
:10070000061208000430F000520851185708A723B9
:100710000800FF305C0784000008CC0005304C075F
:100720004C074C074C07F000840A0430C80000084E
:10073000A723840AF00AC80B972B08000430C800CE
:10074000B6238000F00A840AC80BA02B0800831689
:100750009A0070089B001C1555309D00AA309D0022
:100760009C149C18B12B1C1183120800831670086E
:100770009B001C141A0883120800C223C223C22340
:10078000C2230800C523C5230800FF30C100D62BB3
:100790008030C100D62B4030C100D62B2030C100A4
:1007A000D62B1030C100D62B0230C100FF30C20062
:0A07B000C20BD82BC10BD62B08009A
:084000005700330043004400A7
:02400E00303F41
:10420000CA0017005C002200020050009E001B0044
:104210000000400052003600000000006C006B00FF
:104220000000A0005B009A000000E0008900D600BA
:10423000000080001F0014000100A0005900410090
:104240000100100009007C00010060002900AC00A2
:104250000100E0004400A3000000C8002200560056
:1042600000003800FF004A000000B800CD00330015
:1042700000005800F10006000000000000000000EF
:00000001FF
